:100000000C942A000C9445000C9445000C94450077
:100010000C9445000C9445000C9445000C9445004C
:100020000C9445000C9445000C9445000C9445003C
:100030000C9445000C9445000C9445000C9445002C
:100040000C9445000C9445000C9445000C9445001C
:100050000C94450011241FBECFE5D8E0DEBFCDBF14
:1000600010E0A0E6B0E0E0E8F3E002C005900D92F9
:10007000A036B107D9F710E0A0E6B0E001C01D92AC
:10008000A036B107E1F70C948D000C94000087E8CE
:1000900086B908951CBE13BC8DE783BF85BD089546
:1000A000877087B9369A3699FECF84B195B1089595
:1000B000882311F46CBF0895813009F0089563BD61
:1000C00008950895882321F488B3836088BB089538
:1000D00088B38C7F88BB08950895CF93DF93EC019C
:1000E0001816190654F460E0862F0E94580081E02B
:1000F0000E9462006C2F81E00BC060E081E00E94F2
:10010000580080E00E9462008C2F8195682F80E06B
:100110000E945800DF91CF910895CFE5D8E0DEBF6F
:10012000CDBF1ABA8FEF87BB14BA80E881BB0E949B
:1001300047000E944A0080E00E945000AA2797FDD5
:10014000A095BA2FBC01CD010E942501DC01CB0195
:1001500020E030E040E05FE3BC01CD010E946F0190
:10016000DC01CB0120E030E040E853E4BC01CD01EC
:100170000E94C500DC01CB01BC01CD010E94080139
:10018000DC01CB010E946D00D6CF5058192E84D0CF
:1001900001D06AC0BA176207730784079507B1F1E7
:1001A00088F40EF410940B2EBA2FA02D062E622F79
:1001B000202D072E732F302D082E842F402D092E31
:1001C000952F502DFF275523B9F0591B49F0573E65
:1001D00098F0469537952795A795F0405395C9F720
:1001E00076F0BA0F621F731F841F30F487957795DE
:1001F0006795B795F040939517FA0F2E0895BF1B9A
:10020000BB27BA0B620B730B840BF6CFDEF661C013
:1002100097FB4ED09F3738F0FEE9F91B982F872FB8
:10022000762F6B2F05C052C0969587957795679569
:10023000F150D0F73EF490958095709561957F4F81
:100240008F4F9F4F0895E89403C097FB0EF4F3DFA0
:10025000B62F672F782F892F9EE9002405C09A9525
:10026000BB0F661F771F881F11249923A1F08823D5
:10027000B2F79F3F59F0BB0F48F421F4002011F46E
:1002800060FF04C06F5F7F4F8F4F9F4F881F979510
:10029000879597F908951AC0052E092607FA440F85
:1002A000551F5F3F79F0AA27A51708F051E0479541
:1002B000880F991F9F3F31F0BB27B91708F091E0D5
:1002C000879508959F919F91112457C0662777279E
:1002D000882799270895592F482F372F262FDCDF9D
:1002E00001D0C2CF992339F0552329F09F575F578A
:1002F000950F13F4CAF1EDCF91589F3FE1F3A62F6C
:1003000000241124BB2766275527F8E0A69520F482
:10031000020E131EB41F651F220F331F441F551FEB
:10032000FA95A1F7F8E0E72F7727F8E0E69520F4B3
:10033000130EB41F651F7A1F330F441F551FAA1FCA
:10034000FA95A1F7F82F8827F69520F4B40F651FCA
:100350007A1F8E1F440F551FAA1FEE1FFF23A1F700
:1003600088231AF4939539F408C0000C111CBB1FA4
:10037000661F771F881F012808959FEF80EC08955E
:00000001FF
